:1000000000308A00642A00000030A1001F08C339B4
:1000100021049F000D30A000A00B0C289F149F18F6
:100020000F281E08A601A500260CA300250CA2007F
:10003000A30CA20CA30CA20CA30CA20C2208AB00D4
:100040000430A1001F08C33921049F000D30A00017
:10005000A00B28289F149F182B281E08A801A70072
:10006000280CA300270CA200A30CA20CA30CA20C2A
:10007000A30CA20C2208AC000C30A1001F08C3394D
:1000800021049F000D30A000A00B44289F149F184E
:1000900047281E08AA01A90000344C30840000083B
:1000A00003195F280230A100A001A00B5528A10B65
:1000B00054289730A000A00B5B28800B52280034F6
:1000C000CC014C08293C031C742805150830A000FD
:1000D000A00B6828000005110330A000A00B6E28BB
:1000E00000000000CC0A612800340830CD02031C57
:1000F00084284D3084000310800C000803198428E4
:1001000082280000800B81280034CC014C08143C6C
:10011000031C992805150830A000A00B8D280000AD
:1001200005110330A000A00B932800000000CC0AAA
:1001300086280034AA08031DA2282908DB3C031CDA
:10014000A228851600340130B500B601B701B80009
:10015000B900C9010420051185122F0BB228BA017C
:10016000BB01B828AF08031DB828BA010130BB0095
:100170002B080F3C031DBE280E30AB00CB014B08F3
:10018000033C031CDB280F30AB052B08B200013009
:10019000B205320BD2284B080A3C353E84000130B0
:1001A0008000D7284B080A3C353E840080010310AC
:1001B000AB0CCB0ABF28851DEA280B30CB004B08BF
:1001C0000E3C031CE92835304B0784008001CB0A24
:1001D000DF2810292C08053C031CFD280B30CB0020
:1001E0004B080E3C031CFC2835304B0784000130C3
:1001F00080008516CB0AF02810292C08093C03182A
:1002000010290B30CB004B080D3C031C0E29353058
:100210004B07840080018516CB0A03290130C300F7
:100220002C08063C031C2E290130C4002C08023C7B
:10023000031C1E29C5010130C6002D292C08043CD1
:10024000031C26290130C500C6012D292C08063CB7
:10025000031C2D290130C500C6004929C4012C0802
:10026000083C031C3629C501C60149292C080A3C53
:10027000031C3E29C5010130C60049292C080C3C4D
:10028000031C46290130C500C60149290130C500BB
:10029000C600B1010330CB004B080F3C031C5F29A3
:1002A00035304B0784000310000DB10701304B07B8
:1002B000353E84000008B1070230CB074C29460BBD
:1002C00064290310460DB1070330B105B108031DC1
:1002D0006D290130C700C8008129310B7329C7017E
:1002E0000130C80081293108023C031D7B290130FF
:1002F000C700C80181293108033C031D8129C701BA
:10030000C801CB014B08143C031C9E2935304B0718
:100310008400000B942960200330CC00C630CD004F
:100320007520CC0B8E299C2985200330CC00C6304B
:10033000CD007520CC0B9729CB0A822905119A2074
:10034000DC30CC004D20C62A4D08A1014C02031818
:10035000AC294C08A000B829A0010830CE00CC0D73
:10036000A00D4D0820020318A000A10DCE0BAF294F
:10037000EA290420051185122D0BC5290130AE078D
:100380002E08033C031DC529AD012F0BC929B60159
:10039000CB290130B6002C08073C031CD329B70138
:1003A0000130B800DD292C080A3C0318DB29013094
:1003B000B700B801DD29B701B801AF08031DE52971
:1003C0002D0BE5290130B700B8002B08CC00033015
:1003D000CD00A4292108AB000730AB050430CB00C9
:1003E0004B08063C031C082A2B08B2000130B2055A
:1003F000320B002A35304B07840001308000042A7C
:1004000035304B07840080010310AB0CCB0AF02978
:100410002F0B102A2D0B102AB9010130BA00BB0096
:10042000B1010130CB004B08063C031C1E2A3530BD
:100430004B0784000008B107CB0A132A0130B1052D
:10044000B108031D252ABC01272A0130BC00CB01BD
:100450004B08023C031C2F2A6020CB0A282A0130BB
:10046000CC004D200130CB004B08063C031C532A26
:1004700035304B078400000B492A60200130CC0046
:100480004D200230CC00F830CD007520CC0B432A33
:10049000512A60200230CC00F830CD007520CC0B02
:1004A0004C2ACB0A342ABC08031D582A8520592A15
:1004B000602005119A203C30CC004D202F0B632A80
:1004C0001430CC004D20CA2A84011F3083051F132D
:1004D00083161F149F141F159F15073083129F004A
:1004E000703083168F001B30650083121F13831634
:1004F0001F149F141F119F151F129F161F13831285
:100500009F131F14703083168F00831285120420EE
:10051000851D8E2A0130B400B301912AB401013047
:10052000B300A608031D982A25080C3C03189C2A32
:10053000AF010330B000A02A0130AF000230B0009C
:10054000A608031DA72A2508043C0318A92A04208D
:10055000A02ACA0130084A020318B82A8516FA30C0
:10056000CC004D208512FA30CC004D20CA0AAA2AB0
:10057000330BC32A85160230CB00FA30CC004D2055
:10058000CB0BBD2A8512340BC72AA328C32A330BF1
:08059000CB2AB929C72A630038
:02400E00C43FAD
:00000001FF
